:100000000C9434000C944F000C944F000C944F004F
:100010000C944F000C944F000C944F000C944F0024
:100020000C944F000C944F000C944F000C944F0014
:100030000C944F000C944F000C944F000C944F0004
:100040000C944F000C944F000C944F000C944F00F4
:100050000C944F000C944F000C944F000C944F00E4
:100060000C944F000C944F0011241FBECFEFD4E02E
:10007000DEBFCDBF11E0A0E0B1E0E6E6F2E002C0F5
:1000800005900D92AE30B107D9F711E0AEE0B1E0C6
:1000900001C01D92AF30B107E1F70C94CA000C9477
:1000A0000000209A08959C01832F99278093C50012
:1000B0002093C4001092C00088E98093C1008EE0B4
:1000C0008093C2000895BC0120E0161617063CF488
:1000D000CB016AE070E00E940C012F5FF6CF822F07
:1000E000992708950F931F93CF93DF93EC018B0112
:1000F0000E946300282F3327C9010197A2F0FC0159
:10010000E00FF11FCE016AE070E00E940C01805DFB
:1001100080833197CE016AE070E00E940C01EB0110
:10012000E017F1077CF7200F311FF9011082C80199
:10013000DF91CF911F910F910895FC018081882359
:1001400041F08091C00085FFFCCF81918093C60073
:10015000F5CF089510927C0080EC80937A0008958A
:1001600080937C0080917A008F7E80937A008091CA
:100170007A00806480937A0080917A0084FFFCCFBB
:1001800020917800809179009927982F8827820FF5
:10019000911D0895C9EFD4E0DEBFCDBF0E9451008C
:1001A00083E390E00E9453000E94AA00289A80E016
:1001B0000E94B0008C0181E00E94B0007C0182E0CE
:1001C0000E94B0006C0180E091E00E949D00BE01A1
:1001D0006F5F7F4FC8010E9472000E949D0083E004
:1001E00091E00E949D00BE016F5F7F4FC7010E949A
:1001F00072000E949D0087E091E00E949D00BE0178
:100200006F5F7F4FC6010E9472000E949D008BE0CD
:1002100091E00E949D00CBCF97FB092E07260AD0C4
:1002200077FD04D00CD006D000201AF470956195AB
:100230007F4F0895F6F7909581959F4F0895AA1BDB
:10024000BB1B51E107C0AA1FBB1FA617B70710F0C1
:10025000A61BB70B881F991F5A95A9F780959095F3
:06026000BC01CD01089570
:0E026600783A0020793A00207A3A000D0A001A
:00000001FF
